:020000040000FA
:040000003BEF00F0E2
:0800080040D0076E010E026EEC
:100010000850065C02E10750055C040ED8B0010EE2
:10002000D8B4020E0214D8A4010E1200086A076E9A
:10003000FF0E0726082200D0D8A01200030E066E7D
:10004000E70E02D8F5D7066AFE0F056E000000D055
:1000500000D0E86A065AD8A01200050600D000D0E9
:10006000F5D7066A086AD1DF04E008C006F007C0C9
:1000700005F005501200F86A006A7F0EAF6E240E7C
:10008000AC6E900EAB6E000196D09EAA1BD0060EF1
:10009000AB1412E1E1CF38F0E2CF39F03A2A15EE95
:1000A00000F03A50E126000EE222AECFE7FF38C062
:1000B000E1FF39C0E2FF1100AE50AE50AB98AB8803
:1000C00011000FD0F2A40DD0F294235202E1245279
:1000D00002E0364A372A2450231002E1366A376A92
:1000E000110011003A503B5C14E03B2AE9CF05F0C7
:1000F000EACF06F005EE00F03B50E926000EEA22BA
:10010000EF50056E05C0E9FF06C0EAFFD880120077
:1001100004D0E868056ED8A0120012000D683A50AD
:100120003B5C16E03B2AE9CF05F0EACF06F005EE8E
:1001300000F03B50E926000EEA22EFCF0DF0EF5021
:10014000056E05C0E9FF06C0EAFFD880120006D0A0
:10015000E868056ED8A00DC0DEFF12000DC0DEFFFE
:1001600012000D683B28036E046A0436045204E151
:1001700003503A5CD8B412003B2A05EE00F03B5025
:10018000E926000EEA22EF500D6E12003A6A3B6A31
:100190009D8AF28EF28C12009D9A05EE00F0000E00
:1001A000EE6AE82EFDD73A6A3B6A9D8A12009EA845
:1001B000FED7AD6E1200400E926EE00E936EC00E32
:1001C000946E93908A9093928A9293948A94939641
:1001D0008A9693988A98939A8A9A929A899A9298E8
:1001E0008998929689969294899492928992929003
:1001F000899094908B9094968B9694988B98949ADF
:100200008B9A94928B9294948B9406D07EEC08F007
:1002100008D0AEEC0BF005D089EC10F002D0FCEC6D
:1002200014F0640E03DFB2DFB7DF170ED56ED76AA6
:10023000D66AF294F28AD58E92EC07F068EC07F059
:10024000949A8B8A4FDF0D6EC20E0D5C07E3FE0E93
:100250000D5C02E3B0D102D0126AADD10DAE28D050
:10026000126A810E0D5C05E10DC012F0136814686E
:100270001ED0910E0D5C05E10DC012F015681668D8
:1002800016D0A10E0D5C05E10DC012F017681868BC
:100290000ED0B10E0D5C05E10DC012F019681A68A0
:1002A00006D0C10E0D5C03E10DC012F01B6883D1B6
:1002B000125202E180D17FD1810E125C3AE1132803
:1002C00003E10DC013F033D00DC014F0240E135C05
:1002D00004E372D913686FD129D0070E135C26E2AC
:1002E00000EEBCF01350EB50056E05081DE3FA6AF2
:1002F000D8900536FA360536FA36100E0526030E66
:10030000FA220500030EFE6E280EFD6E0550F96EF2
:1003100097EF04F09AEF04F09DEF04F0A0EF04F0E3
:10032000A3EF04F0A6EF04F0136845D1136843D19E
:1003300042D1910E125CD8A41AD1152803E10DC048
:1003400015F013D10DC016F0165233E1240E155CD2
:1003500007E315C013F016C014F02ED9136827D088
:10036000070E155C24E200EEBCF01550EB50056E54
:1003700005081DE3FA6AD8900536FA360536FA36CE
:10038000960E0526030EFA220500030EFE6EAE0E33
:10039000FD6E0550F96E97EF04F09AEF04F09DEFB3
:1003A00004F0A0EF04F0A3EF04F0A6EF04F015684A
:1003B00002D1180E155C2AE2070E155C24E200EE4D
:1003C000BCF01550EB50056E05081DE3FA6AD89095
:1003D0000536FA360536FA36EE0E0526030EFA22F3
:1003E0000500040EFE6E060EFD6E0550F96ECDEF93
:1003F00004F0D0EF04F0D3EF04F0D6EF04F0D9EF1F
:1004000004F0DCEF04F01568D6D0AAD0240E155CF9
:1004100033E200EE3CF01550EB50056E0B0829E37B
:10042000FA6AD8900536FA360536FA36420E0526AF
:10043000040EFA220500040EFE6E720EFD6E0550CB
:10044000F96E12EF08F01BEF08F024EF08F02DEF23
:1004500008F036EF08F03FEF08F048EF08F051EFF2
:1004600008F05AEF08F063EF08F06CEF08F075EF52
:1004700008F01568A0D074D07F0E155CD8B06ED08F
:10048000240E155C0E6E01EE3BF0D8900E34E9267A
:10049000000EEA22EECF03F0EFCF04F0035203E1A7
:1004A0000452D8B45AD001EE3BF0D8900E34E9266D
:1004B000000EEA22EECF2CF0EFCF2DF00F0E2D1410
:1004C000256E00EEC3F02550EB50036E03520EE193
:1004D00000EEC3F025502CC0EBFF2D380F0B2F6E14
:1004E00002EEABF00E50EB502E6E37D001EEF3F073
:1004F000D8900E34E926000EEA22EECF03F0EFCFBB
:1005000004F0035202E1045226E001EEF3F0D89029
:100510000E34E926000EEA22EECF2CF0EFCF2DF0BC
:100520000F0E2D14256E00EEC3F02550EB50036E18
:1005300003520EE100EEC3F025502CC0EBFF2D3826
:100540000F0B2F6E03EE07F00E50EB502E6E02D005
:10055000156831D002D015682ED002D015682BD086
:100560000C0E255CD8A08DD8156825D024D0A10EFE
:10057000125C0AE1172803E10DC017F003D00DC08B
:1005800018F01DDA18D017D0B10E125C0BE1192843
:1005900003E10DC019F004D00DC01AF06DEC05F0A8
:1005A0000AD009D0C10E125C06E11B2804E10DC07F
:1005B0001BF04AEC05F046D6106A0C0E105C0AE2FD
:1005C00000EECFF01050EB50036E1350035C02E0CE
:1005D000102AF3E10C0E105CD8B051D0800E10241C
:1005E000306E730E135C07E23050E1DD240EDFDD68
:1005F0001450DDDD0BD0B00E1024306E3050D7DD3E
:100600007B0ED7EC00F0000ED7EC00F0F36800EEA4
:10061000CFF01050F3CFEBFFF36A00EEC3F01050B1
:10062000F3CFEBFF1050056E0B0829E3FA6AD89060
:100630000536FA360536FA364E0E0526060EFA222D
:100640000500060EFE6E7E0EFD6E0550F96E73EF10
:1006500004F076EF04F079EF04F07CEF04F07FEF24
:1006600004F082EF04F085EF04F088EF04F08BEFE4
:1006700004F08EEF04F091EF04F094EF04F01368AF
:10068000120001EE17F02550EB50036E035213E1F8
:10069000B00E2524306E3050D7EC00F0450ED7EC6C
:1006A00000F0400ED7EC00F0400EF36E01EE17F0B4
:1006B0002550F3CFEBFF900E2524306EB00E25248D
:1006C000316E00EEC3F02550EB50326E2F5213E125
:1006D0003050D7EC00F0240ED7EC00F01650D7ECD9
:1006E00000F03150D7EC00F0160ED7EC00F032508D
:1006F000D7EC00F057D0010E2F5C13E13050D7EC4F
:1007000000F0300ED7EC00F01650D7EC00F031506E
:10071000D7EC00F0160ED7EC00F03250D7EC00F01A
:1007200041D0020E2F5C13E13050D7EC00F03C0EAC
:10073000D7EC00F01650D7EC00F03150D7EC00F0B9
:10074000160ED7EC00F03250D7EC00F02BD0030E91
:100750002F5C13E13050D7EC00F0480ED7EC00F0DE
:100760001650D7EC00F03150D7EC00F0160ED7EC55
:1007700000F03250D7EC00F015D0040E2F5C12E1DF
:100780003050D7EC00F0540ED7EC00F01650D7ECF8
:1007900000F03150D7EC00F0160ED7EC00F03250DC
:1007A000D7EC00F000EEDBF02550EB50036E2E503E
:1007B000035C11E0B00E2524306E3050D7EC00F011
:1007C000180ED7EC00F02E50D7EC00F000EEDBF066
:1007D00025502EC0EBFF28C005F0165031EC00F07C
:1007E000336E01EE0BF02550EB50036ED8900334BE
:1007F000106E1050FE08116E10C005F0335031EC31
:1008000000F0266E11C005F0335031EC00F0276E79
:1008100001EE23F0255016C0EBFF00EEE7F0255067
:10082000EB50036E2650035C11E0B00E2524306EB1
:100830003050D7EC00F0030ED7EC00F02650D7EC88
:1008400000F000EEE7F0255026C0EBFF00EEF3F0DD
:100850002550EB50036E2750035C11E0B00E2524A9
:10086000306E3050D7EC00F0040ED7EC00F027507B
:10087000D7EC00F000EEF3F0255027C0EBFF00EEC0
:10088000CFF0255015C0EBFF2550056E0B0829E36E
:10089000FA6AD8900536FA360536FA36B20E0526CB
:1008A000080EFA220500080EFE6EE20EFD6E0550DF
:1008B000F96EA9EF04F0ACEF04F0AFEF04F0B2EF83
:1008C00004F0B5EF04F0B8EF04F0BBEF04F0BEEFB6
:1008D00004F0C1EF04F0C4EF04F0C7EF04F0CAEF76
:1008E00004F01568120093908A90120093928A92F5
:1008F000120093948A94120093968A961200939809
:100900008A981200939A8A9A1200929A899A1200EF
:1009100092988998120092968996120092948994DE
:1009200012009292899212009290899012009490F3
:100930008B90120094968B96120094988B981200CC
:10094000949A8B9A120094928B92120094948B94A6
:10095000120093908A80120093928A8212009394DC
:100960008A84120093968A86120093988A881200CD
:10097000939A8A8A1200929A898A12009298898898
:1009800012009296898612009294898412009292A3
:100990008982120092908980120094908B801200BC
:1009A00094968B86120094988B881200949A8B8A66
:1009B000120094928B82120094948B8412000E6A1F
:1009C0000C0E0E5C0AE200EECFF00E50EB50036E00
:1009D0001750035C02E00E2AF3E10C0E0E5CD8B057
:1009E000120000EEC3F00E50EB50036E0352D8B469
:1009F0004FD028C005F0185031EC00F0336E01EEF6
:100A00000BF00E50EB50036ED8900334106E105064
:100A1000FE08116E10C005F0335031EC00F0266E68
:100A200011C005F0335031EC00F0276E00EEE7F016
:100A30000E50EB50036E2650035C11E0B00E0E24F6
:100A4000306E3050D7EC00F0030ED7EC00F026509B
:100A5000D7EC00F000EEE7F00E5026C0EBFF00EE02
:100A6000F3F00E50EB50036E2750035C11E0B00E14
:100A70000E24306E3050D7EC00F0040ED7EC00F0AE
:100A80002750D7EC00F000EEF3F00E5027C0EBFF3C
:100A9000176812001B50056E04081BE3FA6AD89011
:100AA0000536FA360536FA36BE0E05260A0EFA2245
:100AB00005000A0EFE6ED20EFD6E0550F96E7EEF39
:100AC00008F07EEF08F0AEEF0BF089EF10F0FCEFCE
:100AD00014F01B6812001D681200070E195CD8A4E0
:100AE00068D01AC028F00E6A0C0E0E5CD8B05FD029
:100AF00000EEC3F00E50EB50036E0352D8B454D046
:100B000001EE23F00E50EB50036E28C005F00350A9
:100B100031EC00F0336E01EE0BF00E50EB50036E33
:100B2000D8900334106E1050FE08116E10C005F0FE
:100B3000335031EC00F0266E11C005F0335031EC2B
:100B400000F0276E00EEE7F00E50EB50036E2650DB
:100B5000035C11E0B00E0E24306E3050D7EC00F084
:100B6000030ED7EC00F02650D7EC00F000EEE7F0D3
:100B70000E5026C0EBFF00EEF3F00E50EB50036E6C
:100B80002750035C11E0B00E0E24306E3050D7ECCD
:100B900000F0040ED7EC00F02750D7EC00F000EE88
:100BA000F3F00E5027C0EBFF0E2AD8A49DD7E9D052
:100BB000E8D0170E195C0DE10E6A0C0E0E5C07E210
:100BC00001EE0BF00E501AC0EBFF0E2AF6E1D9D061
:100BD000D8D01E0E195C0BE32A0E195C08E21E0E1B
:100BE000195C01EE0BF01AC0EBFFCBD0CAD0320E6D
:100BF000195C1DE33E0E195C1AE2320E195C00EE20
:100C0000FFF01AC0EBFFCE0E19240B6E0C6AFF0E1C
:100C10000C22B00E0B24306E3050D7EC00F0140EC6
:100C2000D7EC00F01A50D7EC00F0ABD0AAD0400EB1
:100C3000195C1AE11A5202E1296A02D0400E296EAB
:100C4000106A0C0E105C0EE2B00E1024306E3050A4
:100C5000D7EC00F0400ED7EC00F02950D7EC00F0B4
:100C6000102AEFE18ED08DD0410E195C16E11AC02A
:100C70002AF0106A0C0E105C0EE2B00E1024306EDA
:100C80003050D7EC00F0410ED7EC00F02A50D7ECF2
:100C900000F0102AEFE175D074D0420E195C1FE10C
:100CA0001A5202E170D819D0106A0C0E105C15E2CD
:100CB000B00E1024306E3050D7EC00F0450ED7EC5B
:100CC00000F0400ED7EC00F0400EF36E01EE17F08E
:100CD0001050F3CFEBFF102AE8E153D052D0500E62
:100CE000195C1DE35C0E195C1AE2B00E19240B6E40
:100CF0000C6AFF0E0C22B00E0B24306E3050D7EC75
:100D000000F0180ED7EC00F01A50D7EC00F0500E9F
:100D1000195C00EEDBF01AC0EBFF33D032D0640E6A
:100D2000195C2BE3700E195C28E2640E195C106EDE
:100D300000EEC3F01050EB50036E03521CE01A5249
:100D40001AE0410E1A5C17E201EE2FF010501AC0A3
:100D5000EBFFB00E1024306E3050D7EC00F0160EC2
:100D6000D7EC00F01A50D7EC00F000EEC3F01050B2
:100D70001AC0EBFF06D005D004D07B0E195CD8B4A6
:100D800002D819681200B00ED7EC00F07B0ED7EC39
:100D900000F0000ED7EC00F0B10ED7EC00F07B0EA7
:100DA000D7EC00F0000ED7EC00F0B20ED7EC00F05C
:100DB0007B0ED7EC00F0000ED7EC00F0B30ED7ECB2
:100DC00000F07B0ED7EC00F0000ED7EC00F0B40E74
:100DD000D7EC00F07B0ED7EC00F0000ED7EC00F063
:100DE000B50ED7EC00F07B0ED7EC00F0000ED7EC80
:100DF00000F0B60ED7EC00F07B0ED7EC00F0000E42
:100E0000D7EC00F0B70ED7EC00F07B0ED7EC00F07B
:100E1000000ED7EC00F0B80ED7EC00F07B0ED7EC4C
:100E200000F0000ED7EC00F0B90ED7EC00F07B0E0E
:100E3000D7EC00F0000ED7EC00F0BA0ED7EC00F0C3
:100E40007B0ED7EC00F0000ED7EC00F0BB0ED7EC19
:100E500000F07B0ED7EC00F0000ED7EC00F0939082
:100E60008A9093928A9293948A9493968A9693986E
:100E70008A98939A8A9A929A899A9298899892963D
:100E80008996929489949292899292908990949062
:100E90008B9094968B9694988B98949A8B9A949224
:100EA0008B9294948B94236A246A106A0C0E105CC3
:100EB0000EE2F36A00EEC3F01050F3CFEBFFF368DD
:100EC00000EECFF01050F3CFEBFF102AEFE112004D
:100ED000BC69BD6B010EBE6F020EBF6F030EC06F0B
:100EE000040EC16F050EC26F0E6A800E0E5C08E222
:100EF000F36800EE3CF00E50F3CFEBFF0E2AF5E165
:100F0000180E0E6E240E0E5C0AE2180E0E5C036EB6
:100F100000EE3CF00E5003C0EBFF0E2AF3E1236A13
:100F2000246A1200106A0C0E105CD8B076D0B00E95
:100F30001024306E400EF36E01EE17F01050F3CF18
:100F4000EBFF400EF36E01EE0BF01050F3CFEBFF12
:100F5000400E1024326E00EEFFF0105032C0EBFF56
:100F6000400EF36E00EEDBF01050F3CFEBFF400EBF
:100F7000F36E00EEE7F01050F3CFEBFF400EF36E90
:100F800000EEF3F01050F3CFEBFFF36A00EEC3F086
:100F90001050F3CFEBFF3050D7EC00F0450ED7ECFC
:100FA00000F0400ED7EC00F0140ED7EC00F03250F9
:100FB000D7EC00F0160ED7EC00F0010ED7EC00F0E5
:100FC000180ED7EC00F0400ED7EC00F0030ED7EC73
:100FD00000F0400ED7EC00F0040ED7EC00F0400E0D
:100FE000D7EC00F0060E16EC00F0296A0F0E2A6E00
:100FF0003050D7EC00F0400ED7EC00F02950D7EC81
:1010000000F0410ED7EC00F02A50D7EC00F0040EAF
:1010100016EC00F0102AD8A486D7400E266E276E54
:10102000286E1200900ED7EC00F0180ED7EC00F0EE
:101030001650D7EF00F0910ED7EC00F0180ED7EC59
:1010400000F01650D7EF00F0920ED7EC00F0180E1B
:10105000D7EC00F01650D7EF00F0930ED7EC00F06D
:10106000180ED7EC00F01650D7EF00F0940ED7EC26
:1010700000F0180ED7EC00F01650D7EF00F0950EE8
:10108000D7EC00F0180ED7EC00F01650D7EF00F0B8
:10109000960ED7EC00F0180ED7EC00F01650D7EFF4
:1010A00000F0970ED7EC00F0180ED7EC00F01650B9
:1010B000D7EF00F0980ED7EC00F0180ED7EC00F048
:1010C0001650D7EF00F0990ED7EC00F0180ED7ECC1
:1010D00000F01650D7EF00F09A0ED7EC00F0180E83
:1010E000D7EC00F01650D7EF00F09B0ED7EC00F0D5
:1010F000180ED7EC00F01650D7EF00F0106A5C0E17
:10110000105C10E2400EF36E02EEABF01050F3CF25
:10111000EBFF400EF36E03EE07F01050F3CFEBFF42
:10112000102AEDE1106A130E105C0BE201EEF3F0F1
:10113000D8901034E926000EEA22EE6AEF6A102AEF
:10114000F2E1010E01013B6F3C6B3D6F3E6F3F6F63
:10115000020E406F010E416F030E426F010E436F8E
:10116000040E446F010E456F050E466F010E476F6A
:10117000060E486F010E496F070E4A6F010E4B6F46
:10118000080E4C6F010E4D6F090E4E6F010E4F6F22
:101190000A0E506F010E516F0B0E526F020E536FFD
:1011A000546B556F010E566F020E576F586F596F83
:1011B000030E5A6F020E5B6F040E5C6F020E5D6FC2
:1011C000050E5E6F020E5F6F060E606F020E616F9E
:1011D000070E626F030E0201196F1A6B020E0101F6
:1011E000636F080E646F030E02011B6F010E1C6F0C
:1011F000020E0101656F090E666F030E02011D6F7D
:10120000020E1E6F0101676F0A0E686F030E020166
:101210001F6F206F020E0101696F0B0E6A6F030EC4
:101220000201216F040E226F01016B6F6C6B030EC4
:101230000201236F050E246F040E01016D6F010E74
:101240006E6F030E0201256F060E266F040E01015C
:101250006F6F020E706F030E0201276F070E286F6B
:10126000040E0101716F030E726F0201296F080EE7
:101270002A6F040E0101736F746F030E02012B6F4E
:10128000090E2C6F040E0101756F050E766F030EAB
:1012900002012D6F0A0E2E6F040E0101776F060EEC
:1012A000786F030E02012F6F0B0E306F040E0101D9
:1012B000796F070E7A6F060E0201316F326B040EE2
:1012C00001017B6F080E7C6F060E0201336F010E69
:1012D000346F040E01017D6F090E7E6F060E020150
:1012E000356F020E366F040E01017F6F0A0E806F9C
:1012F000060E0201376F030E386F040E0101816F75
:101300000B0E826F060E0201396F040E3A6F080E43
:101310000101836F846B060E02013B6F050E3C6F6B
:10132000080E0101856F010E866F060E02013D6FEA
:101330003E6F080E0101876F020E886F060E0201D4
:101340003F6F070E406F080E0101896F030E8A6F11
:10135000060E0201416F080E426F01018B6F040EF1
:101360008C6F060E0201436F090E446F080E0101D7
:101370008D6F050E8E6F060E0201456F0A0E466FC9
:10138000080E01018F6F060E906F0201476F0B0E62
:10139000486F080E0101916F070E926F0C0E02014B
:1013A000496F4A6B080E0101936F946F0C0E020196
:1013B0004B6F010E4C6F080E0101956F090E966F71
:1013C0000C0E02014D6F020E4E6F080E0101976F59
:1013D0000A0E986F0C0E02014F6F030E506F080E2D
:1013E0000101996F0B0E9A6F0C0E0201516F040EE2
:1013F000526F100E01019B6F9C6B0C0E0201536F1C
:10140000050E546F100E01019D6F010E9E6F0C0EA4
:101410000201556F060E566F100E01019F6F020EEE
:10142000A06F0C0E0201576F070E586F100E0101CE
:10143000A16F030EA26F0C0E0201596F080E5A6FB6
:10144000100E0101A36F040EA46F0C0E02015B6F5E
:10145000090E5C6F100E0101A56F050EA66F0C0E34
:1014600002015D6F0A0E5E6F100E0101A76F060E7E
:10147000A86F0C0E02015F6F0B0E606F100E010162
:10148000A96F070EAA6F180E0201616F626B100E32
:101490000101AB6F080EAC6F180E0201636F010EF5
:1014A000646F100E0101AD6F090EAE6F180E0201D0
:1014B000656F020E666F100E0101AF6F0A0EB06FFE
:1014C000180E0201676F030E686F100E0101B16FF5
:1014D0000B0EB26F180E0201696F040E6A6F200EB8
:1014E0000101B36FB46B180E02016B6F050E6C6FC8
:1014F000200E0101B56F010EB66F180E02016D6F5F
:10150000060E6E6F200E0101B76F020EB86F180E37
:1015100002016F6F070E706F200E0101B96F030E8D
:10152000BA6F180E0201716F080E726F200E010162
:10153000BB6F040EBC6F180E0201736F090E746F3F
:10154000200E0101BD6F050EBE6F180E0201756FF2
:101550000A0E766F200E0101BF6F060EC06F180EC7
:101560000201776F0B0E786F200E0101C16F070E1D
:10157000C26F300E0201796F7A6B200E0101C36FCA
:10158000080EC46F300E02017B6F010E7C6F200EBF
:101590000101C56F090EC66F300E02017D6F020E8C
:1015A0007E6F200E0101C76F0A0EC86F300E020158
:1015B0007F6F030E806F200E0101C96F0B0ECA6F83
:1015C000300E0201816F040E826F400E0101CB6F5D
:1015D000CC6B300E0201836F050E846F400E01014B
:1015E000CD6F010ECE6F300E0201856F060E866F35
:1015F000400E0101CF6F020ED06F300E0201876FD7
:10160000070E886F400E0101D16F030ED26F300EAE
:101610000201896F080E8A6F400E0101D36F040E1C
:10162000D46F300E02018B6F090E8C6F400E0101DA
:10163000D56F050ED66F300E02018D6F0A0E8E6FBC
:10164000400E0101D76F060ED86F300E02018F6F6A
:101650000B0E906F400E0101D96F070EDA6F300E3E
:101660000201916F100E926F400E0101DB6F080EA8
:10167000DC6F300E0201936F110E946F400E01016A
:10168000DD6F090EDE6F300E0201956F120E966F40
:10169000400E0101DF6F0A0EE06F300E0201976FFE
:1016A000130E986F400E0101E16F0B0EE26F300ECA
:1016B0000201996F140E9A6F400E0101E36F100E34
:1016C000E46F300E02019B6F150E9C6F400E0101FE
:1016D000E56F110EE66F300E02019D6F160E9E6FC4
:1016E000400E0101E76F120EE86F300E02019F6F8E
:1016F000170EA06F400E0101E96F130EEA6F300E56
:101700000201A16F180EA26F400E0101EB6F140EC3
:10171000EC6F300E0201A36F190EA46F400E010191
:10172000ED6F150EEE6F300E0201A56F1A0EA66F4B
:10173000400E0101EF6F160EF06F300E0201A76F21
:101740001B0EA86F400E0101F16F170EF26F300EE5
:101750000201A96F200EAA6F00011200106A5C0E30
:10176000105C10E2400EF36E02EEABF01050F3CFBF
:10177000EBFF400EF36E03EE07F01050F3CFEBFFDC
:10178000102AEDE1106A130E105C0BE201EEF3F08B
:10179000D8901034E926000EEA22EE6AEF6A102A89
:1017A000F2E1010E01013B6F3C6B400E0201AB6F99
:1017B000010E01013D6F3E6F400E0201AC6F010E44
:1017C00001013F6F020E406F400E0201AD6F010E2E
:1017D0000101416F030E426F400E0201AE6F010E18
:1017E0000101436F040E446F400E0201AF6F010E02
:1017F0000101456F050E466F400E0201B06F010EEC
:101800000101476F060E486F400E0201B16F010ED5
:101810000101496F070E4A6F400E0201B26F010EBF
:1018200001014B6F080E4C6F400E0201B36F010EA9
:1018300001014D6F090E4E6F400E0201B46F010E93
:1018400001014F6F0A0E506F400E0201B56F010E7D
:101850000101516F0B0E526F400E0201B66F020E66
:101860000101536F546B3E0E0201B76F020E01016E
:10187000556F010E566F400E0201B86F020E010146
:10188000576F586F400E0201B96F020E0101596F78
:10189000030E5A6F3C0E0201BA6F020E01015B6F1C
:1018A000040E5C6F410E0201BB6F020E01015D6F01
:1018B000050E5E6F430E0201BC6F020E01015F6FE9
:1018C000060E606F420E0201BD6F020E0101616FD4
:1018D000070E626F3F0E0201BE6F030E196F1A6B87
:1018E000420E03011A6F020E0101636F080E646F4E
:1018F000420E0201BF6F030E1B6F010E1C6F460EDE
:1019000003011B6F020E0101656F090E666F410E28
:101910000201C06F030E1D6F020E1E6F460E030103
:101920001C6F020E0101676F0A0E686F470E0201FD
:10193000C16F030E1F6F206F430E03011D6F020E58
:101940000101696F0B0E6A6F490E0201C26F030E2F
:10195000216F040E226F490E03011E6F040E010158
:101960006B6F6C6B410E0201C36F030E236F050E8C
:10197000246F4C0E03011F6F040E01016D6F010EE9
:101980006E6F4C0E0201C46F030E256F060E266F9C
:101990004C0E0301206F040E01016F6F020E706F79
:1019A0004E0E0201C56F030E276F070E286F4A0EF9
:1019B0000301216F040E0101716F030E726F4B0E54
:1019C0000201C66F296B2A6B400E0301226F040EC1
:1019D0000101736F746F530E0201C76F2B6B2C6B79
:1019E000400E0301236F040E0101756F050E766F23
:1019F000550E0201C86F2D6B2E6B400E0301246F34
:101A0000040E0101776F060E786F580E0201C96F40
:101A10002F6B306B400E0301256F040E0101796FAF
:101A2000070E7A6F560E0201CA6F316B326B400E91
:101A30000301266F040E01017B6F080E7C6F5C0EA4
:101A40000201CB6F336B346B400E0301276F040E22
:101A500001017D6F090E7E6F5D0E0201CC6F356B4B
:101A6000366B400E0301286F070E01017F6F806BFC
:101A7000550E0201CD6F376B386B400E0301296F95
:101A8000040E0101816F0A0E826F2C0E0201CE6FCF
:101A9000050E396F060E3A6F2D0E03012A6F040EE4
:101AA0000101836F0B0E846F3B0E0201CF6F3B6B06
:101AB0003C6B03012B6F060E0101856F050E866FCF
:101AC000410E0201D06F080E3D6F3E6B3F0E0301C9
:101AD0002C6F050E0101876F090E886F420E0201FF
:101AE000D16F060E3F6F406F460E03012D6F050E3E
:101AF0000101896F0A0E8A6F450E0201D26F090E2D
:101B0000416F426B4E0E03012E6F070E01018B6F6A
:101B1000050E8C6F430E0201D36F060E436F090E44
:101B2000446F400E03012F6F080E01018D6F050EEB
:101B30008E6F400E0201D46F060E456F0A0E466F7F
:101B4000400E0301306F080E01018F6F060E906F7B
:101B5000400E0201D56F060E476F0B0E486F400E08
:101B60000301316F080E0101916F070E926F400E55
:101B70000201D66F0C0E496F4A6B400E0301326FA3
:101B8000090E0101936F040E946F400E0201D76F8E
:101B90000C0E4B6F010E4C6F400E0301336F080E9D
:101BA0000101956F070E966F440E0201D86F0A0E61
:101BB0004D6F030E4E6F3C0E0301346F070E010193
:101BC000976F0A0E986F410E0201D96F0C0E4F6F7E
:101BD000030E506F400E0301356F0D0E0101996F1A
:101BE0009A6B3C0E0201DA6F0B0E516F030E526FAF
:101BF0003F0E0301366F100E01019B6F9C6B400E70
:101C00000201DB6F0C0E536F050E546F400E030183
:101C1000376F090E01019D6F080E9E6F3F0E020186
:101C2000DC6F0C0E556F030E566F3C0E0301386FC0
:101C3000100E01019F6F070EA06F400E0201DD6FB5
:101C40000C0E576F070E586F400E0301396F100EC0
:101C50000101A16F030EA26F400E0201DE6F0C0E98
:101C6000596F080E5A6F400E03013A6F100E0101B2
:101C7000A36F040EA46F400E0201DF6F0C0E5B6FAA
:101C8000090E5C6F400E03013B6F110E0101A56F41
:101C9000A66B3F0E0201E06F0C0E5D6F060E5E6FCD
:101CA000400E03013C6F0E0E0101A76F040EA86FDA
:101CB0003D0E0201E16F0F0E5F6F030E606F460E67
:101CC00003013D6F0D0E0101A96F060EAA6F3D0EB7
:101CD0000201E26F180E616F626B400E03013E6FEE
:101CE000100E0101AB6F080EAC6F400E0201E36FE6
:101CF000180E636F010E646F400E03013F6F0F0EED
:101D00000101AD6F050EAE6F440E0201E46F140EBB
:101D1000656F666B400E0301406F100E0101AF6FDF
:101D20000A0EB06F400E0201E56F180E676F030ECA
:101D3000686F400E0301416F100E0101B16F0B0E71
:101D4000B26F400E0201E66F180E696F040E6A6FE3
:101D5000400E0301426F0F0E0101B36F070EB46F07
:101D60003C0E0201E76F130E6B6F030E6C6F430E98
:101D70000301436F160E0101B56F010EB66F400EE1
:101D80000201E86F180E6D6F060E6E6F400E0301B4
:101D9000446F170E0101B76F010EB86F490E0201B3
:101DA000E96F180E6F6F070E706F400E0301456FDD
:101DB000180E0101B96F040EBA6F440E0201EA6FEA
:101DC000180E716F080E726F400E0301466F160EEB
:101DD0000101BB6F030EBC6F400E0201EB6F180ECA
:101DE000736F746B3C0E0301476F1B0E0101BD6FD7
:101DF000BE6B3E0E0201EC6F100E756F090E766F12
:101E00003F0E0301486F150E0101BF6F050EC06F35
:101E1000420E0201ED6F190E776F020E786F410EC0
:101E20000301496F170E0101C16F040EC26F3E0E10
:101E30000201EE6F1A0E796F020E7A6F470E0301E0
:101E40004A6F130E0101C36F080EC46F410E0201E9
:101E5000EF6F1E0E7B6F7C6B3C0E03014B6F160EFB
:101E60000101C56F060EC66F3F0E0201F06F300E06
:101E70007D6F020E7E6F400E03014C6F200E01013C
:101E8000C76F0A0EC86F400E0201F16F300E7F6FF0
:101E9000030E806F400E03014D6F150E0101C96FD7
:101EA000080ECA6F3E0E0201F26F190E816F050E09
:101EB000826F430E03014E6F400E0101CB6FCC6B5E
:101EC0000201F36F300E836F050E846F400E030125
:101ED0004F6F1E0E0101CD6F030ECE6F3D0E02013E
:101EE000F46F300E856F060E866F400E0301506F43
:101EF000160E0101CF6F090ED06F4A0E0201F56F69
:101F00001A0E876F060E886F3C0E0301516F180E74
:101F10000101D16F080ED26F400E0201F66F1B0E49
:101F2000896F060E8A6F410E0301526F400E010148
:101F3000D36F040ED46F400E0201F76F1C0E8B6F2F
:101F4000060E8C6F480E0301536F400E0101D56FD2
:101F5000050ED66F400E0201F86F300E8D6F0A0E1F
:101F60008E6F400E0301546F190E0101D76F090ED9
:101F7000D86F450E0201F96F300E8F6F0B0E906F08
:101F8000400E0301556F170E0101D96F0B0EDA6F6A
:101F9000420E0201FA6F300E916F100E926F400EDA
:101FA0000301566F1E0E0101DB6F070EDC6F400E42
:101FB0000201FB6F300E936F110E946F400E030100
:101FC000576F1C0E0101DD6F0A0EDE6F420E02011B
:101FD000FC6F1F0E956F070E966F410E0301586F31
:101FE0001E0E0101DF6F080EE06F400E0201FD6F53
:101FF000200E976F070E986F410E0301596F400E28
:102000000101E16F0B0EE26F3B0E0201FE6F300E1D
:10201000996F140E9A6F400E03015A6F4D0E010115
:10202000E36F0B0EE46F470E0201FF6F300E9B6FE4
:10203000150E9C6F400E03015B6F0101E56F110EE1
:10204000E66F400E0301006F300E02019D6F160E09
:102050009E6F400E03015C6F200E0101E76F090EB9
:10206000E86F3B0E0301016F300E02019F6F170EE8
:10207000A06F400E03015D6F0101E96F130EEA6F5F
:10208000400E0301026F300E0201A16F180EA26F05
:10209000400E03015E6F0101EB6F140EEC6F400EFA
:1020A0000301036F300E0201A36F190EA46F400EDF
:1020B00003015F6F0101ED6F150EEE6F400E03011E
:1020C000046F300E0201A56F1A0EA66F400E0301B9
:1020D000606F0101EF6F160EF06F400E0301056F88
:1020E000300E0201A76F1B0EA86F400E0301616F37
:1020F0000101F16F170EF26F400E0301066F300EF3
:102100000201A96F200EAA6F400E0301626F000149
:102110001200106A5C0E105C22E2400EF36E02EEBA
:10212000ABF01050F3CFEBFF400EF36E03EE07F071
:102130001050F3CFEBFF01EEF3F0D8901034E92606
:10214000000EEA22EE6AEF6A01EE3BF0D8901034FE
:10215000E926000EEA22EE6AEF6A102ADBE1010EA0
:1021600001013B6F3C6B400E0201AB6F010E0101A0
:102170003D6F3E6F400E0201AC6F010E01013F6FDB
:10218000020E406F400E0201AD6F010E0101416F62
:10219000030E426F400E0201AE6F010E0101436F4C
:1021A000040E446F400E0201AF6F010E0101456F36
:1021B000050E466F400E0201B06F010E0101476F20
:1021C000060E486F400E0201B16F010E0101496F0A
:1021D000070E4A6F400E0201B26F010E01014B6FF4
:1021E000080E4C6F400E0201B36F010E01014D6FDE
:1021F000090E4E6F400E0201B46F010E01014F6FC8
:102200000A0E506F400E0201B56F010E0101516FB1
:102210000B0E526F400E0201B66F020E0101536F9A
:10222000546B420E0201B76F020E0101556F010E91
:10223000566F440E0201B86F020E0101576F586FBE
:102240003F0E0201B96F020E0101596F030E5A6F62
:10225000430E0201BA6F020E01015B6F040E5C6F48
:102260001E0E0201BB6F020E01015D6F050E5E6F57
:10227000360E0201BC6F020E01015F6F060E606F29
:10228000310E0201BD6F020E0101616F070E626F18
:10229000420E0201BE6F030E196F1A6B480E030146
:1022A0001A6F020E0101636F080E646F3E0E020189
:1022B000BF6F030E1B6F010E1C6F4A0E03011B6FD5
:1022C000020E0101656F090E666F3C0E0201C06FC0
:1022D000020E0101676F0A0E686F420E0201C16FA4
:1022E000030E1F6F206F350E03011D6F020E0101DB
:1022F000696F0B0E6A6F480E0201C26F030E010177
:102300006B6F050E6C6F450E0201C36F040E236FD9
:10231000246B470E03011F6F040E01016D6F010E48
:102320006E6F4C0E0201C46F030E01016F6F070E3A
:10233000706F4B0E0201C56F030E0101716F080E25
:10234000726F400E0201C66F040E296F030E2A6FD2
:10235000440E0301226F030E0101736F090E746FA7
:102360003C0E0201C76F050E2B6F2C6B4E0E030146
:10237000236F050E0101756F010E766F4A0E020183
:10238000C86F030E0101776F0B0E786F420E0201CA
:10239000C96F040E2F6F060E306F4C0E0301256FB0
:1023A000050E0101796F030E7A6F480E0201CA6FA4
:1023B000040E01017B6F080E7C6F4A0E0201CB6F89
:1023C000060E01017D6F020E7E6F370E0201CC6F8B
:1023D000050E01017F6F060E806F520E0201CD6F58
:1023E000060E0101816F040E826F470E0201CE6F4F
:1023F000080E0101836F846B460E0201CF6F080E39
:102400000101856F010E866F3A0E0201D06F090E31
:102410003D6F3E6B150E03012C6F070E0101876F98
:10242000040E886F560E0201D16F060E0101896FEE
:10243000080E8A6F340E0201D26F080E01018B6FF5
:10244000050E8C6F090E0201D36F080E436F030E49
:10245000446F6B0E03012F6F080E01018D6F040E88
:102460008E6F710E0201D46F0A0E456F020E466F19
:10247000210E0301306F060E01018F6F0A0E906F5F
:102480005C0E0201D56F0A0E0101916F040E926F6E
:102490001B0E0201D66F0B0E496F020E4A6F2E0EF5
:1024A0000301326F070E0101936F0B0E946F200E24
:1024B0000201D76F0A0E0101956F050E966F460E49
:1024C0000201D86F0C0E4D6F020E4E6F440E0301C9
:1024D000346F0C0E0101976F040E986F0D0E020100
:1024E000D96F0B0E4F6F040E506F550E0301356FF1
:1024F000080E0101996F0B0E9A6F3F0E0201DA6F01
:102500000A0E516F080E526F130E0301366F100E34
:1025100001019B6F010E9C6F1A0E0201DB6F0F0E03
:10252000536F010E546F520E0301376F100E0101ED
:102530009D6F020E9E6F0A0E0201DC6F0F0E556F2B
:10254000020E566F410E0301386F0F0E01019F6F8F
:10255000040EA06F130E0201DD6F0E0E576F040EF6
:10256000586F4B0E0301396F0D0E0101A16F060E5E
:10257000A26F560E0201DE6F110E0101A36F030E52
:10258000A46F340E0201DF6F0C0E0101A56F0B0E5C
:10259000A66F090E0201E06F0B0E5D6F5E6F540EA9
:1025A00003013C6F0D0E0101A76F0A0EA86F2D0EDF
:1025B0000201E16F110E0101A96F060EAA6F3F0E15
:1025C0000201E26F0F0E0101AB6F0A0EAC6F1C0E21
:1025D0000201E36F0E0E636F0A0E646F580E030163
:1025E0003F6F110E0101AD6F090EAE6F0A0E0201B1
:1025F000E46F100E656F090E666F420E0301406FA7
:10260000100E0101AF6F0B0EB06F070E0201E56FE8
:102610000F0E676F0B0E686F3A0E0301416F100EBD
:102620000101B16F0B0EB26F400E0201E66F180E82
:10263000696F040E6A6F400E0301426F0F0E0101B5
:10264000B36F070EB46F3C0E0201E76F130E6B6F92
:10265000030E6C6F430E0301436F160E0101B56F3D
:10266000010EB66F400E0201E86F180E6D6F060E78
:102670006E6F400E0301446F170E0101B76F010E1C
:10268000B86F490E0201E96F180E6F6F070E706F79
:10269000400E0301456F180E0101B96F040EBA6FA9
:1026A000440E0201EA6F180E716F080E726F400E31
:1026B0000301466F160E0101BB6F030EBC6F400E87
:1026C0000201EB6F180E736F746B3C0E0301476FC2
:1026D0001B0E0101BD6FBE6B3E0E0201EC6F100EB2
:1026E000756F090E766F3F0E0301486F150E0101DD
:1026F000BF6F050EC06F420E0201ED6F190E776FAE
:10270000020E786F410E0301496F170E0101C16F70
:10271000040EC26F3E0E0201EE6F1A0E796F020EAA
:102720007A6F470E03014A6F130E0101C36F080E43
:10273000C46F410E0201EF6F1E0E7B6F7C6B3C0E6F
:1027400003014B6F160E0101C56F060EC66F3F0EDB
:102750000201F06F300E7D6F020E7E6F400E03019E
:102760004C6F200E0101C76F0A0EC86F400E0201A8
:10277000F16F300E7F6F030E806F400E03014D6FBF
:10278000150E0101C96F080ECA6F3E0E0201F26FED
:10279000190E816F050E826F430E03014E6F400EBE
:1027A0000101CB6FCC6B0201F36F300E836F050E0E
:1027B000846F400E03014F6F1E0E0101CD6F030E9B
:1027C000CE6F3D0E0201F46F300E856F060E866FE0
:1027D000400E0301506F160E0101CF6F090ED06F2E
:1027E0004A0E0201F56F1A0E876F060E886F3C0EB7
:1027F0000301516F180E0101D16F080ED26F400E08
:102800000201F66F1B0E896F060E8A6F410E0301DF
:10281000526F400E0101D36F040ED46F400E0201BF
:10282000F76F1C0E8B6F060E8C6F480E0301536FF3
:10283000400E0101D56F050ED66F400E0201F86FF4
:10284000300E8D6F0A0E8E6F400E0301546F190EFD
:102850000101D76F090ED86F450E0201F96F300ED6
:102860008F6F0B0E906F400E0301556F170E010115
:10287000D96F0B0EDA6F420E0201FA6F300E916FB4
:10288000100E926F400E0301566F1E0E0101DB6F9A
:10289000070EDC6F400E0201FB6F300E936F110EBE
:1028A000946F400E0301576F1C0E0101DD6F0A0E7D
:1028B000DE6F420E0201FC6F1F0E956F070E966FC2
:1028C000410E0301586F1E0E0101DF6F080EE06F0D
:1028D000400E0201FD6F200E976F070E986F410E9C
:1028E0000301596F400E0101E16F0B0EE26F3B0EC9
:1028F0000201FE6F300E996F140E9A6F400E0301A5
:102900005A6F4D0E0101E36F0B0EE46F470E02018B
:10291000FF6F300E9B6F150E9C6F400E03015B6FB7
:102920000101E56F110EE66F400E0301006F300EDE
:1029300002019D6F160E9E6F400E03015C6F200E0C
:102940000101E76F090EE86F3B0E0301016F300EC6
:1029500002019F6F170EA06F400E03015D6F010112
:10296000E96F130EEA6F400E0301026F300E020191
:10297000A16F180EA26F400E03015E6F0101EB6F95
:10298000140EEC6F400E0301036F300E0201A36FB3
:10299000190EA46F400E03015F6F0101ED6F150E5C
:1029A000EE6F400E0301046F300E0201A56F1A0E88
:1029B000A66F400E0301606F0101EF6F160EF06FFE
:1029C000400E0301056F300E0201A76F1B0EA86FAA
:1029D000400E0301616F0101F16F170EF26F400E9F
:1029E0000301066F300E0201A96F200EAA6F400E80
:1029F0000301626F00011200106A5C0E105C10E2AD
:102A0000400EF36E02EEABF01050F3CFEBFF400E32
:102A1000F36E03EE07F01050F3CFEBFF102AEDE159
:102A2000106A130E105C0BE201EEF3F0D890103434
:102A3000E926000EEA22EE6AEF6A102AF2E1010EA0
:102A400001013B6F3C6B400E0201AB6F010E0101B7
:102A50003D6F3E6F400E0201AC6F010E01013F6FF2
:102A6000020E406F400E0201AD6F010E0101416F79
:102A7000030E426F400E0201AE6F010E0101436F63
:102A8000040E446F400E0201AF6F010E0101456F4D
:102A9000050E466F400E0201B06F010E0101476F37
:102AA000060E486F400E0201B16F010E0101496F21
:102AB000070E4A6F400E0201B26F010E01014B6F0B
:102AC000080E4C6F400E0201B36F010E01014D6FF5
:102AD000090E4E6F400E0201B46F010E01014F6FDF
:102AE0000A0E506F400E0201B56F010E0101516FC9
:102AF0000B0E526F400E0201B66F020E0101536FB2
:102B0000546B3E0E0201B76F020E0101556F010EAC
:102B1000566F400E0201B86F020E0101576F586FD9
:102B2000400E0201B96F020E0101596F030E5A6F78
:102B30003C0E0201BA6F020E01015B6F040E5C6F66
:102B4000410E0201BB6F020E01015D6F050E5E6F4B
:102B5000430E0201BC6F020E01015F6F060E606F33
:102B6000420E0201BD6F020E0101616F070E626F1E
:102B70003F0E0201BE6F030E196F1A6B420E030166
:102B80001A6F020E0101636F080E646F420E02019C
:102B9000BF6F030E1B6F010E1C6F460E03011B6FF0
:102BA000020E0101656F090E666F410E0201C06FD2
:102BB000030E1D6F020E1E6F460E03011C6F020EE8
:102BC0000101676F0A0E686F470E0201C16F030EA5
:102BD0001F6F206F430E03011D6F020E0101696F0D
:102BE0000B0E6A6F490E0201C26F030E216F040EB5
:102BF000226F490E03011E6F040E01016B6F6C6B97
:102C0000410E0201C36F030E236F050E246F4C0E9D
:102C100003011F6F040E01016D6F010E6E6F4C0EEC
:102C20000201C46F030E256F060E266F4C0E0301C2
:102C3000206F040E01016F6F020E706F4E0E0201C5
:102C4000C56F030E276F070E286F4A0E0301216F11
:102C5000040E0101716F030E726F4B0E0201C66FFD
:102C6000296B2A6B400E0301226F040E0101736F62
:102C7000746F530E0201C76F2B6B2C6B400E030158
:102C8000236F040E0101756F050E766F550E02015C
:102C9000C86F2D6B2E6B400E0301246F040E0101D3
:102CA000776F060E786F580E0201C96F2F6B306B6D
:102CB000400E0301256F040E0101796F070E7A6F34
:102CC000560E0201CA6F316B326B400E0301266F44
:102CD000040E01017B6F080E7C6F5C0E0201CB6F4E
:102CE000336B346B400E0301276F040E01017D6FBF
:102CF000090E7E6F5D0E0201CC6F356B366B400E98
:102D00000301286F070E01017F6F806B550E0201D2
:102D1000CD6F376B386B400E0301296F040E010134
:102D2000816F0A0E826F2C0E0201CE6F050E396F75
:102D3000060E3A6F2D0E03012A6F040E0101836FF8
:102D40000B0E846F3B0E0201CF6F3B6B3C6B03019C
:102D50002B6F060E0101856F050E866F410E020175
:102D6000D06F080E3D6F3E6B3F0E03012C6F050EBA
:102D70000101876F090E886F420E0201D16F060EA6
:102D80003F6F406F460E03012D6F050E0101896FE5
:102D90000A0E8A6F450E0201D26F090E416F426B17
:102DA0004E0E03012E6F070E01018B6F050E8C6F07
:102DB000430E0201D36F060E436F090E446F400E9F
:102DC00003012F6F080E01018D6F050E8E6F400EEF
:102DD0000201D46F060E456F0A0E466F400E0301C6
:102DE000306F080E01018F6F060E906F400E0201CA
:102DF000D56F060E476F0B0E486F400E0301316F03
:102E0000080E0101916F070E926F400E0201D66FFE
:102E10000C0E496F4A6B400E0301326F090E01011F
:102E2000936F040E946F400E0201D76F0C0E4B6F20
:102E3000010E4C6F400E0301336F080E0101956FB8
:102E4000070E966F440E0201D86F0A0E4D6F030EE7
:102E50004E6F3C0E0301346F070E0101976F0A0E8F
:102E6000986F410E0201D96F0C0E4F6F030E506F19
:102E7000400E0301356F0D0E0101996F9A6B3C0EE8
:102E80000201DA6F0B0E516F030E526F3F0E0301FA
:102E9000366F100E01019B6F9C6B400E0201DB6FC1
:102EA0000C0E536F050E546F400E0301376F090E61
:102EB00001019D6F080E9E6F3F0E0201DC6F0C0E2C
:102EC000556F030E566F3C0E0301386F100E010153
:102ED0009F6F070EA06F400E0201DD6F0C0E576F43
:102EE000070E586F400E0301396F100E0101A16FDC
:102EF000030EA26F400E0201DE6F0C0E596F080E1A
:102F00005A6F400E03013A6F100E0101A36F040EB9
:102F1000A46F400E0201DF6F0C0E5B6F090E5C6F39
:102F2000400E03013B6F110E0101A56FA66B3F0E12
:102F30000201E06F0C0E5D6F060E5E6F400E030126
:102F40003C6F0E0E0101A76F040EA86F3D0E02012B
:102F5000E16F0F0E5F6F030E606F460E03013D6F52
:102F60000D0E0101A96F060EAA6F3D0E0201E26F60
:102F7000180E616F626B400E03013E6F100E01016F
:102F8000AB6F080EAC6F400E0201E36F180E636F5B
:102F9000010E646F400E03013F6F0F0E0101AD6F14
:102FA000050EAE6F440E0201E46F140E656F666B82
:102FB000400E0301406F100E0101AF6F0A0EB06F9B
:102FC000400E0201E56F180E676F030E686F400E2A
:102FD0000301416F100E0101B16F0B0EB26F400E75
:102FE0000201E66F180E696F040E6A6F400E03014E
:102FF000426F0F0E0101B36F070EB46F3C0E02015A
:10300000E76F130E6B6F030E6C6F430E0301436F7C
:10301000160E0101B56F010EB66F400E0201E86F8A
:10302000180E6D6F060E6E6F400E0301446F170E83
:103030000101B76F010EB86F490E0201E96F180E5A
:103040006F6F070E706F400E0301456F180E010180
:10305000B96F040EBA6F440E0201EA6F180E716F59
:10306000080E726F400E0301466F160E0101BB6F12
:10307000030EBC6F400E0201EB6F180E736F746B82
:103080003C0E0301476F1B0E0101BD6FBE6B3E0E70
:103090000201EC6F100E756F090E766F3F0E030183
:1030A000486F150E0101BF6F050EC06F420E020181
:1030B000ED6F190E776F020E786F410E0301496FA5
:1030C000170E0101C16F040EC26F3E0E0201EE6FBA
:1030D0001A0E796F020E7A6F470E03014A6F130EB4
:1030E0000101C36F080EC46F410E0201EF6F1E0E87
:1030F0007B6F7C6B3C0E03014B6F160E0101C56F9D
:10310000060EC66F3F0E0201F06F300E7D6F020E8D
:103110007E6F400E03014C6F200E0101C76F0A0E37
:10312000C86F400E0201F16F300E7F6F030E806F8B
:10313000400E03014D6F150E0101C96F080ECA6FD5
:103140003E0E0201F26F190E816F050E826F430E63
:1031500003014E6F400E0101CB6FCC6B0201F36F88
:10316000300E836F050E846F400E03014F6F1E0EED
:103170000101CD6F030ECE6F3D0E0201F46F300ED4
:10318000856F060E866F400E0301506F160E01010B
:10319000CF6F090ED06F4A0E0201F56F1A0E876FBE
:1031A000060E886F3C0E0301516F180E0101D16F9E
:1031B000080ED26F400E0201F66F1B0E896F060ECD
:1031C0008A6F410E0301526F400E0101D36F040E4E
:1031D000D46F400E0201F76F1C0E8B6F060E8C6FC2
:1031E000480E0301536F400E0101D56F050ED66FD7
:1031F000400E0201F86F300E8D6F0A0E8E6F400E7A
:103200000301546F190E0101D76F090ED86F450ED7
:103210000201F96F300E8F6F0B0E906F400E03019D
:10322000556F170E0101D96F0B0EDA6F420E0201B6
:10323000FA6F300E916F100E926F400E0301566FB1
:103240001E0E0101DB6F070EDC6F400E0201FB6FEB
:10325000300E936F110E946F400E0301576F1C0ECA
:103260000101DD6F0A0EDE6F420E0201FC6F1F0EC0
:10327000956F070E966F410E0301586F1E0E0101E8
:10328000DF6F080EE06F400E0201FD6F200E976F9A
:10329000070E986F410E0301596F400E0101E16F57
:1032A0000B0EE26F3B0E0201FE6F300E996F140E93
:1032B0009A6F400E03015A6F4D0E0101E36F0B0E22
:1032C000E46F470E0201FF6F300E9B6F150E9C6F6F
:1032D000400E03015B6F0101E56F110EE66F400EBA
:1032E0000301006F300E02019D6F160E9E6F400E9F
:1032F00003015C6F200E0101E76F090EE86F3B0EC2
:103300000301016F300E02019F6F170EA06F400E78
:1033100003015D6F0101E96F130EEA6F400E0301B7
:10332000026F300E0201A16F180EA26F400E030152
:103330005E6F0101EB6F140EEC6F400E0301036F23
:10334000300E0201A36F190EA46F400E03015F6FD0
:103350000101ED6F150EEE6F400E0301046F300E8C
:103360000201A56F1A0EA66F400E0301606F0101E6
:10337000EF6F160EF06F400E0301056F300E020165
:10338000A76F1B0EA86F400E0301616F0101F16F63
:10339000170EF26F400E0301066F300E0201A96F87
:1033A000200EAA6F400E0301626F00011200FFD7CA
:020000040030CA
:03000100460F0E99
:020005008D80EC
:060008000FC00FE00F40E5
:00000001FF
